:020000040800F2
:10000000201D0020A90100081D150008410C000852
:1000100000000000000000000000000000000000E0
:100020000000000000000000000000005D1C00084F
:1000300000000000000000001F1500085D1D000802
:10004000BB010008BB010008BB010008BB010008A0
:10005000BB010008BB010008BB010008BB01000890
:1000600000000000BB010008BB010008BB01000844
:10007000BB010008BB010008BB0100080000000034
:10008000BB010008BB01000800000000611E000861
:10009000951E00081D1F0008411F0008BB01000835
:1000A000BB010008BB010008BB010008951F000848
:1000B00025200008000000000000000000000000F3
:1000C000BB01000800000000BB01000800F002F8BE
:1000D00000F03EF80CA030C8083824182D18671E10
:1000E000A246AB4654465D46AC4201D100F030F822
:1000F0007E460F3EB6460FCC0126334200D0FB1A97
:100100003343A246AB461847984A0000B84A00005D
:10011000103A02D378C878C1FAD8520701D330C850
:1001200030C101D504680C60704700000023002432
:1001300000250026103A01D378C1FBD8520700D31E
:1001400030C100D50B6070471FB51FBD10B510BD85
:1001500000F090FB1146FFF7F7FF02F07DFD00F085
:10016000A8FB03B4FFF7F2FF03BC00F007FC00009C
:1001700070B505460C46164602E00FCC0FC5103E82
:10018000102EFAD2082E02D303CC03C5083E042E4B
:1001900007D301CC01C5361F03E021782970641C08
:1001A0006D1C761EF9D270BD07488047074800478E
:1001B000FEE7FEE7FEE7FEE7FEE7FEE70448054947
:1001C000054A064B70470000711D0008CD0000086D
:1001D00020150020201D00202019002020190020BB
:1001E000F8B5042A2CD3830712D00B78491C03706E
:1001F000401C521E83070BD00B78491C0370401C17
:10020000521E830704D00B78491C0370401C521EF9
:100210008B079B0F05D0C91ADF002023DE1B08C9FE
:100220000AE0FFF7A5FFF8BD1D4608C9FD401C46C2
:10023000B4402C4310C0121F042AF5D2F308C91A87
:10024000521EF0D40B78491C0370401C521EEAD495
:100250000B78491C0370401C012AE4D40978017012
:10026000F8BD7047704770470246C80FC00781430A
:100270004B0030B54B405B009B0D20D01923DB06B3
:10028000C91801231B05994220DB0324A407042578
:100290001346AB400BD3002B04D1EB0613409B005D
:1002A000E34204D401246407002312195941FF23B7
:1002B0001B0599420BD2C9000143500F09E0CB0244
:1002C00004D501430803024305D0054830BDFF2192
:1002D000C905084330BD084607210905884330BDDC
:1002E0000000C07FF0B58B4C0F09254689B0BD4397
:1002F0007BD01D092646AE43FAD00E465E4027400D
:10030000F60F3E43254071D024012142FBD0FF244B
:10031000AD19A4042D1B039501252D05DB02DB0A75
:10032000C9022B43C90A29431E010901040F130FF7
:10033000050121431701880B820391432D098C4647
:10034000A90B1E438A039543B30B9A0396433F09B7
:10035000BA0B9403A74302962E467E430497B646F3
:100360004E19D7190C460196544305977E43371B07
:100370007646BF1B3601B646BE0B3619009676464A
:10038000BC043719009C01D3641C00946400002F46
:1003900001D001263443029E049F754366467E4386
:1003A0000496760034196E0034190094029C019E64
:1003B0001C196643751BAE46069465464519059C97
:1003C00005956C43594375460891691A0191049E3D
:1003D00001465143A41B0491611A009C0791E10658
:1003E00005D061090122114302E072E06EE061096B
:1003F000089D00272C0A2D066918049D7C412A0AB5
:100400002D066918019D6241AC0DAD026D18544175
:10041000079A910D920255196141029A6446584318
:100420005443069B059A5A43121A131B9A0E9B01BA
:100430005B187A41010B0005C3185141220A2006BE
:1004400044195A419A4200D2491C0120400281427B
:1004500003D315230226F64302E014230326F643B2
:100460002020C51AA9401746AF40DA400A4320466B
:100470000399D8400914731819055118039A384381
:10048000D2075140AC4009D00122944006D300224B
:10049000401C5141002C01D1400840001E4A9342AB
:1004A00012D3012203989206904207DB05204007F1
:1004B00009181A480143C012414004E003204007D4
:1004C0000818C10FC907002009B0F0BD0020F107CE
:1004D000FAE705180C464C4111486D42A04115D36E
:1004E00094181A465A410E48644290410ED3012096
:1004F0004A004005824209D35A00824206D359403D
:10050000C90F084AC90700201143DDE7002006494A
:10051000DAE700000000FF07FE070000FFFFFF7F93
:100520000000E0FF0000F07F0000F87F0121C90516
:100530000123411842001B06D3185B0E0AD0C110DC
:100540000722D206891840075242D14201D55200F3
:1005500089187047090208D50146002A03D0C10F47
:10056000C9070020704710467047420202D00020A1
:1005700002497047072109050143F4E70000F87FAD
:10058000F0B5FF252D04C609C209FF2704462E40F9
:100590000137CB093E4348402A402B400746002AFA
:1005A0006BD0002B69D0AA4267D0AB4265D000283F
:1005B00000DA32460125ED0529432C4309022002C9
:1005C000090AD21A4B0C7F24E31A434C000A7C44DC
:1005D000E35C7D242404121914145B00A2188842E1
:1005E00001D3521C00E0400049420C465C432411F8
:1005F0005C43DB016415E318040A5C43C502200D6B
:100600000C4644436419250A5D432303EC0C0D4654
:10061000654300030019EB184C42A34201D35B1859
:10062000401CD4052018002B07D05B00C91804D348
:10063000401C002901D1400840003F2189048A4222
:1006400009D3002A08DC1106090F04D00321490749
:100650004018C00FC007F0BD0122410012068918E2
:100660007F2252069142F6D205214907C84201D5A0
:100670009010F0BDFF20C005F0BD002F00DA32461B
:100680001648AA4207D2AB4205D21902090E17D06A
:10069000F80FC007F0BDFF2563002D06AB42F9D867
:1006A0004900A942F6D8AB4201D1A942F2D0A942F1
:1006B00001D1002101E061004908D0050843F0BDE7
:1006C0001102090EFBD0FF200243D005F0BD0A46FF
:1006D0000146104654E70000A64200000000C07F1B
:1006E0000102C21504D00123DB071943002A0ADBEB
:1006F0009E239A1A02D40846D0407047FF22410038
:100700001206914201D900207047C017C0437047BC
:100710001F22030C02D10F2200041CD0030E01D1B2
:100720000002083A030F01D10001121F830F01D10B
:100730008000921E002801DB4000521ED205511895
:10074000021251181922904004D3491C002801D1EB
:100750004908490008467047C10FC90700D0404208
:10076000012292071143D3E701218907D0E7000056
:10077000F8B5264C4E00069DA6420AD8A64201D1E5
:10078000002806D15E00A64203D8A6420AD1002A5C
:1007900008D00D242404254233D02946002000F03F
:1007A00090F8F8BD0C461C4311D4994207D0C81AE2
:1007B00002D3EFF30080F8BDEFF30080F8BD801A9C
:1007C00002D3EFF30080F8BDEFF30080F8BD0924F9
:1007D0002407E5008B4207D0581A02D3EFF30080BC
:1007E00006E0EFF3008007E0101A03D3EFF3008078
:1007F000A04303E0EFF30080A043284380F3008888
:10080000F8BD009500F074F8F8BD00000000E0FFAE
:1008100010B5FF231B0644009C421DD84C009C428F
:100820001AD80346124A0B4307D4401A02D3EFF3F7
:10083000008010BDEFF3008010BD081A03D3EFF362
:100840000080904305E0EFF3008001219043C90749
:10085000084380F3008810BD0D231B041A4204D006
:100860001146002000F02DF810BD00F04BF810BD2F
:1008700000000090754600F04DF8AE460500694650
:100880005346C008C000854618B020B5FFF796FC57
:1008900060BCB64600260027C0C5C0C5C0C5C0C5DF
:1008A000C0C5C0C5C0C5C0C5403D490849008D464A
:1008B000704710B50446C046C0462046FFF751FCBD
:1008C00010BDC80212D54803400F002804D0C80349
:1008D000C043012188407047EFF300800001000908
:1008E00003210907084380F3008870470020704700
:1008F00010B500200249029A00F010F810BD000067
:100900000000F87F10B5024800F008F810BD0000A4
:100910000000C07F004870479800002010B50C46CA
:100920001107090F092904D00A290AD008290CD176
:1009300004E011460820FFF7C4FF06E0510606D583
:1009400001E0510601D50120C007214610BDD106A6
:1009500007D501010909CC084907000E0006044328
:1009600009E0410F20024907000A0143200E00065A
:100970001D22D14101430846E7E700000149182044
:10098000ABBEFEE726000200704770B514460D4668
:100990000646200407D0B0B200F006F82870641EA6
:1009A0006D1C761CF5E770BD70B5044600F0D8F8F4
:1009B000A020214DA847214EB047200AA847B047A4
:1009C000E0B2A847B04700F0CBF8A120A847B04755
:1009D000002000F037F9044600F0E2F8204670BD30
:1009E00070B514460D460646200407D02978B0B2EB
:1009F00000F006F8641E6D1C761CF5E770BD000063
:100A0000F8B50C46054600F0ABF8A0200A4EB047FA
:100A10000A4FB847280AB047B847E8B2B047B847C6
:100A20002046B047B84700F0BBF80A20F8BC02BC2B
:100A30008E4600F083B8C046A90C00080D0D0008D2
:100A400080B500F013F800F0B1FF01F0C3F801F039
:100A500019F801F089F800F057FF00F0E5FF00F009
:100A60000DFF80BC01BC864601F042B8F8B50020FD
:100A7000022101F053FB0A2000F060F8664D28794E
:100A8000411973268C5D00F0B1F8844208D17420BE
:100A9000285C00022946743149784018286301E037
:100AA0000120687101240221204601F037FB0A2051
:100AB00000F044F8287941198F5D00F097F88742DB
:100AC00008D17420285C0002294674314978401806
:100AD000686300E06C711320022101F01FFB0A2003
:100AE00000F02CF8287941198E5D00F07FF88642DD
:100AF00008D17420285C00022946743149784018D6
:100B0000A863F8BD6C71F8BD80B5C54841F200011D
:100B100002F05DF8411E884180BDC04674223E4807
:100B200000217E2A02D08154521CFAE78170018094
:100B30007047C0462C4800214170704781B000903A
:100B400003480099016001680029FCD101B0704799
:100B50003C0C002081B00090009801B0704700006C
:100B6000F8B501F0C7F8E44C01262046314602F002
:100B70002AF802252046294602F025F8042738469F
:100B8000FFF7E8FF2046314602F01BF83846FFF732
:100B9000E1FF20462946F8BC04BC964602F011B895
:100BA000F8B501F0A7F8D44C02252046294602F0FA
:100BB00008F801262046314602F003F8042738469B
:100BC000FFF7C8FF2046294601F0FDFF20463146C9
:100BD00001F0F9FF3846F8BC02BC8E46FFF7BABFF9
:100BE000014840787047C046F8000020B0B5401E6C
:100BF0000021094B74240A46CDB2A84204DD5D19D8
:100C00002D5D5219491CF7E70C4801788918407886
:100C10000918FF208843B0BD2401002010B5401EF4
:100C20000021064B0A46CCB2A04203DD1C5D12191E
:100C3000491CF8E7FF20904310BDC046400C00203F
:100C4000FEE70000FEB5009001F04EF800210226FC
:100C5000012001900C46019D07291CD8A64F38465B
:100C60000291314601F0ADFF3046FFF773FF384681
:100C7000314601F0A8FF3846294601F0A8FF274673
:100C800004462846FFF766FF0299601E84417800FB
:100C90000419491CE0E7009810B100F0E7FF01E0FB
:100CA00001F004F8E0B2FEBDFEB5044601F022F802
:100CB00091480226314601F084FF0027012001906F
:100CC000072F1FD860B2002802948B4D284603D40A
:100CD000019901F076FF02E0019901F074FF3046BE
:100CE000094CA0472846314601F06DFF3046A04729
:100CF0002846314601F065FF3046A0477F1C029C24
:100D00006400DDE7FEBDC046550B000870B500F07D
:100D1000EBFF794C0221204601F055FF01252846C2
:100D2000FFF718FF00262046294601F050FF30B19A
:100D3000701CFA2E0646F6D3FFF732FF04E00221BC
:100D4000204601F03EFF0025284670BD00F06AB83D
:100D5000FEB5A94802F080FE0920C60601210191D6
:100D60000025202730462A463B46A44CA0470322B4
:100D70000292A34C304629463B46A04730463946AE
:100D8000A04A90471027304601992A463B469B4C83
:100D9000A04730462946029A3B46994CA047304628
:100DA0003946984A90474027304601992A463B46A3
:100DB000924CA04730462946029A3B46904CA047A9
:100DC000304639468F4A90478027304601992A4657
:100DD0003B468A4CA04730462946029A3B46884CFF
:100DE000A04730463946874A90478348401C02F066
:100DF00033FE854E3046019C21462A4623467F4FCE
:100E0000B84730462946029A23467D4DA8473046CA
:100E100021467C4A03B0F0BC08BC9E461047C04641
:100E200000040048F8B51C4802F016FE1B4F0125CF
:100E30000024724E38462946224642F20003B0474B
:100E40006F4E38462146224642F20003B0473846EC
:100E500042F2000101F0B5FE0F48C01C02F0FCFD9B
:100E6000254E3046294622462B46644FB847304629
:100E7000214622462B46624FB84702273046294674
:100E800022463B465D4DA8473046214622463B461A
:100E90005B4CA047F8BDC0461305000000080048A1
:100EA000F8B5E14CA34D2046A847601CA847601D3B
:100EB000A847114E002401258023504F304621467B
:100EC0002A46B8474023304621462A46B8470920DB
:100ED000C606304621462A4641F20003B84730464E
:100EE00021462A4640F20013B847F24821462A46D6
:100EF00048F20003B847F8BD00140048B0B50D48EB
:100F000002F0AAFDEB4C0121002520462A4640F6BE
:100F1000000301F061FE03222046294640F600034B
:100F200001F079FE204640F60001B0BC04BC9646B4
:100F300001F047BE1205000070470000F0B585B013
:100F4000D94C204602F088FD601C02F085FD092086
:100F5000C40601260227D64D204631463A4648F2BD
:100F60000003A8470021039103220492244D204648
:100F700048F20003A847204648F20001214A904762
:100F8000CC4808250296314601973A462B46C84C74
:100F9000A047C8480399049A2B46194CA047C54C52
:100FA00020462946174A90471025204631463A46A2
:100FB0002B46BF4EB04720462746039E3146049A33
:100FC0002B460F4CA047384629460E4A904720250D
:100FD00038460299019A2B46B54CA047384631460F
:100FE000049A2B46064CA04738462946054A05B0C8
:100FF000F0BC08BC9E46104711050000D92B000824
:10100000172C0008C32B0008000400480C48006897
:1010100040F2E831B0FBF1F0401E010E00D0FEE7D7
:101020000849094A5060094803680B4003218907B1
:101030005918016000209060072010607047C0467A
:1010400010000020FFFFFF0010E000E020ED00E0B6
:10105000F0B587B03648002141600E4601919349B2
:1010600040F210608847344D34492846884703AC25
:101070003349204688474720029020803148059018
:101080000496314A28462146904701272F4A284690
:10109000394600979047142002212D4A90472D4948
:1010A0002846884740F21060401C804988472A4EF5
:1010B00030462249884703AD28462149884702988F
:1010C000288020480590019C0494304629461E4AF9
:1010D0009047304639461D4A90471520032529463A
:1010E0001B4A904730461B49884740F21060801CDD
:1010F0006E498847194E30461049884703AF384635
:101100000F498847164838801648059004943046A1
:1011100039460D4A9047304600990C4A90471620B0
:1011200029460B4A904730460A49884707B0F0BD28
:10113000F8000020593A000800400140F53B000843
:10114000413D0008E7030000693C00081D3D000820
:101150005D3800085F3C0008004401400048014041
:101160001F1C00000F270000FEB502901C20022566
:10117000294602F073FB4C4802F06EFC0920C706BA
:1011800001240426019638462146324601F0EEFC41
:10119000384629462246334601F01EFD00210091C3
:1011A00038462246334601F036FD082638462146A9
:1011B000324601F0DBFC384629462246334601F030
:1011C0000BFD3846009F39462246334601F023FD89
:1011D000164802F041FC164D284602F007FE28464C
:1011E000029902F0D1FD2846394602F079FE2846E0
:1011F00041F2000102F089FE284640F2004102F06F
:101200005AFE2846019902F063FE2846314602F054
:1012100074FE284602F004FE0521284603B0F0BC07
:1012200004BC964602F01ABE11050000110700002A
:1012300000440040F8B51C4C1C4D2046A847641CD7
:101240002046A8472046A8470920C5060126184C75
:101250002846314632463346A04700240327284615
:1012600021463A46334601F0D6FCA04802253146D5
:101270002A4644F200030E4EB0479C4E30462146AB
:101280003A4644F2000301F0C6FC304621462A46A5
:1012900041F20003064CA047304644F20001F8BC7E
:1012A00004BC964601F08FBC11050000593A0008B5
:1012B000D92B000800040048F8B500F017FF0A24F5
:1012C0000F4E2046B04700F0DFFE2046B04700201A
:1012D00002250C4A0C4F2946B8472046B04701204A
:1012E00029460246B8471320084A2946B8472046EF
:1012F000B04700F0E1FEF8BC01BC864600F008B83B
:101300003D0B0008040A00004121000865040000AC
:10131000FEB57020022100F001FF3220FFF70EFC25
:101320006D4E3079811973240D5DFFF75FFC8542A6
:1013300007D17420305C000231467431497840187E
:10134000B0607120022100F0E9FE3220FFF7F6FBC9
:10135000307981190D5DFFF749FC854207D1742072
:10136000305C00023146743149784018F0607220D8
:10137000022100F0D3FE3220FFF7E0FB3079811923
:101380000D5DFFF733FC854207D17420305C00020D
:10139000314674314978401830610221204600F00E
:1013A000BDFE3220FFF7CAFB307981190D5DFFF7D2
:1013B0001DFC854207D17420305C00023146743137
:1013C00049784018706174250221284600F0A6FE75
:1013D0003220FFF7B3FB307981190F5DFFF706FC70
:1013E000874206D1705D0002314674314978401859
:1013F000B0617520022100F091FE3220FFF79EFBC4
:10140000307981190F5DFFF7F1FB874206D1705DDE
:1014100000023146743149784018F061762002218B
:1014200000F07CFE3220FFF789FB307981190F5DD7
:10143000FFF7DCFB874206D1705D00023146743154
:101440004978401830627720022100F067FE322090
:10145000FFF774FB307981190F5DFFF7C7FB8742F7
:1014600006D1705D000231467431497840187062CF
:101470006F20022100F052FE3220FFF75FFB30792F
:1014800081190C5DFFF7B2FB844208D1705D000248
:1014900031467431497840180290B06201E0B06A78
:1014A0000290B068019037460C37BCCF306A00908C
:1014B000716A01988218D21812195219D21900981B
:1014C00010184018401E80B204494140F162029851
:1014D000091A48424841FEBD24010020FFFF0000D8
:1014E000E54840F6000101F070BBC046000400482A
:1014F000094A1018C9B24A07D20F02718A07D20FDF
:1015000042700A07D20FC271CA06D20F82728906D0
:10151000C90F41737047C0460000002070477047F4
:10152000F0B58BB00020B34C0490214640F29012ED
:10153000FFF72BFA0894207808B1042802D3AD49AC
:1015400003200870AC49087040F2F810AB49085805
:101550000A9040F2F4100858099040F2F0100A582E
:1015600040F2EC10085840F2E8140C590B25EE43F9
:10157000019608361827DEB19E498D19697DB9405C
:10158000234604460A9808180A9020461C46697C9F
:10159000B940099BCB180993697BB9408A18697ACD
:1015A000B94008186979B9400C19083F761CE2E780
:1015B00040F2F811914E0A9F775040F2F411099DC4
:1015C000755040F2F011725040F2EC11705040F240
:1015D000E813F4508A4E642C01D3B44201D98749F0
:1015E000CE50642802D38649884204D940F2EC10D8
:1015F0006421824C21508348824204D940F2F01089
:101600007E49804B0B508048854204D940F2F4104B
:101610007A497D4A0A507D48874204D940F2F81041
:1016200076497A4A0A500498032872D004908000C0
:101630007249401840F2BC2142580A9240F28C2470
:101640000259099240F25C25435940F22C27C659B1
:1016500040F2FC128258411803910119029141197C
:101660000591C1190791114640F2FC1280180690AD
:10167000019F08371824E7B108460899CD19D921E8
:10168000695CA1400A9A8A180A92A921695CA14062
:10169000099A8A1809927921695CA140CB184921DD
:1016A000695CA1408E19697EA1400918083C7F1C25
:1016B000E1E7079806600698016005980360099FB6
:1016C000029D2F600A9A039C226064294C4801D332
:1016D000814201D906990860642E01D3864202D95D
:1016E0006420079908604748834202D94548059914
:1016F000086045488742049801D943492960434915
:101700008A4201D9414921600899091D0891401C6C
:101710008AE740F20510374E305C40F2F421374A38
:10172000505040F2F8201018019A911D40F20C130D
:1017300021B17418E45C10C0891CF9E740F218105C
:10174000305C40F21C312D4B585040F2403018189C
:1017500040F21E11711803238BB10D7805600C7BCC
:1017600004630DB1642D01D3012505600CB1642C17
:1017700001D301240463491C001D5B1EECE740F209
:101780002710335C40F264311C4D6B5040F2331033
:10179000305C40F2943428510BB1642B02D3012306
:1017A000164C635008B1642804D340F294300121F0
:1017B000124B195040F2411340F2421440F24315CB
:1017C000B2B111461248861837690A48821840F2A9
:1017D0004010105C0006C019D75C3F043818175D34
:1017E0003F023818525D801830610A460A1DE7E74B
:1017F0000BB0F0BDAC080020000000207C020020EF
:10180000B01E04008038010080B14F0100562183D2
:101810005802002070B5154C8021154E2046B04767
:10182000144D287040212046B04768700920C40636
:10183000204641F20001B047A870204640F2001156
:10184000B047E8700C4848F20001B0472978090118
:1018500001436878C0000843A97889000143E8780B
:1018600042000A431F20904370BDC0460014004848
:101870005F1C0008A20100200004004870B522206F
:10188000022100F04BFC0A20FFF758F9F04E3079A6
:10189000811973228C5CFFF7A9F984420AD1742064
:1018A000305A000400BAFEF75FFFFEF73FFE044621
:1018B0000D4603E00120707100242546F06E0D49AD
:1018C00002F043FE08B90D4A00E00B4A08B90D4B7F
:1018D00000E00B4B20462946FEF704FDFEF7C4FC52
:1018E0003067306D3F21090602F019FE08B900206B
:1018F000306770BD00005C42CFF753E34E62105872
:10190000A59BB43F39B4B83F70B52820032100F03F
:1019100005FC0A20FFF712F9CD4D287941197324EF
:101920000E5DFFF763F986420BD17420285C00043A
:10193000294674314A781202101889784018A8652F
:1019400001E0012068710220014600F0E7FB0A2057
:10195000FFF7F4F8287941190C5DFFF747F9844245
:1019600008D17420285C0002294674314978401857
:10197000E86501E001206871A86DFEF7F5FE0446F8
:10198000286AFEF7F1FE0146204602F0B5FE31213D
:10199000090602F0B1FEB04C214602F0ADFE214630
:1019A000FEF7EEFD2866686670BDC046B0B524201F
:1019B000032100F0B3FB0A20FFF7C0F8A44D2879FB
:1019C000411973228C5CFFF711F984420BD174200A
:1019D000285C0004294674314A781202101889786C
:1019E0004018E86302E001206871E86B010218D436
:1019F000FEF7BAFE0446A868FEF7B6FE014620468A
:101A000002F07AFE0D21890602F076FE924C214604
:101A1000FEF7B6FD214602F06FFE2146FEF7B0FD4F
:101A200000E000202864B0BDB0B52320022100F002
:101A300075FB0A20FFF782F8854D2879411973223A
:101A40008C5CFFF7D3F884420BD17420285A000431
:101A500000BAFEF789FE4121090602F04DFE01465B
:101A600002E00120687100210548FEF789FD044667
:101A7000784902F05FFD00B10024AC66B0BDC046FD
:101A8000647A5A4AB0B52C20042100F047FB0A20A2
:101A9000FFF754F86E4D2879411973228C5CFFF7DB
:101AA000A5F8844203D1686F00BAE86402E001201F
:101AB0006871E86C0121CA070021904200D9C9432E
:101AC0004840FEF751FE04466869FEF74DFE214688
:101AD00002F012FE0321090702F00EFE5E4C2146C1
:101AE00002F00AFE2146FEF74BFD2865B0BDC04658
:101AF00070B52720032100F011FB0A20FFF71EF824
:101B0000534E3079811973228C5CFFF76FF8844251
:101B10000AD17420305C0004314674314A781202D4
:101B200010188978441801E001207071306DFEF7BB
:101B3000FDFC0A4A0A4B02F0E7FC05460120C105FC
:101B40008C4201D90006041B2046FEF70DFE054914
:101B5000FEF716FD05B10020F06670BD3333333358
:101B60003333D33FFEFFFF4AB0B52E20042100F0EF
:101B7000D5FA0A20FEF7E2FF354D28794119732284
:101B80008C5CFFF733F8844203D1686F00BAE864D5
:101B900002E001206871E86C0121CA07002190422F
:101BA00000D9C9434840FEF7DFFD04466869FEF7E7
:101BB000DBFD214602F0A0FD0321090702F09CFD98
:101BC000254C214602F098FD2146FEF7D9FC6865B8
:101BD000B0BDC046B0B52620032100F09FFA0A2010
:101BE000FEF7ACFF1A4D2879411973228C5CFEF781
:101BF000FDFF84420BD17420285C00042946743117
:101C00004A781202101889784018686402E00120AE
:101C10006871686C010218D4FEF7A6FD04462869B5
:101C2000FEF7A2FD0146204602F066FD6921C905C6
:101C300002F062FD0749FEF7A3FC074C214602F0C3
:101C40005BFD2146FEF79CFC00E00020A864B0BDCF
:101C5000240100200000C84200007A44704780B58B
:101C600000F0B5FF411E884180BD000070B52D4CCD
:101C700002250D4E20462946B04700F03BF80121D1
:101C80002046B0472846FEF765FF2046294600F06B
:101C90009AFF2846FEF75EFF20462946324670BC72
:101CA00008BC9E461047C046C32B0008B0B51D4C6B
:101CB00002252046294600F084FF00F01BF8012190
:101CC000204600F080FF2846FEF744FF20462946C4
:101CD00000F079FF2846FEF73DFF20462946B0BCBC
:101CE00004BC964600F06DBF0E48002101230A4651
:101CF00000F072BF70B50B4C00250126204631461E
:101D00002A46334600F068FF032220462946334620
:101D100000F081FF044848F2000170BC04BC964604
:101D200000F04FBF0014004800080048F8B5044612
:101D30000027CE4D084EA7420CD0EB48C15D284687
:101D400002F04EF82846314602F077F80028F9D024
:101D50007F1CF0E7F8BDC046060700000348016895
:101D600011B10168491E01607047C0463C0C00205B
:101D700030B43348026801210A43026002689207C6
:101D8000FCD542682F4B1340436042682E4B1340F2
:101D9000436002682D4B13400360C26A0F239A43CD
:101DA000C262026B40F203139A4302630A04036B9C
:101DB00093430363CA07036B93430363426B8A43F2
:101DC00042630022826002680A430260204B0222C2
:101DD00004685D1E9D4202D214402B46F8D0036871
:101DE0009B0700D4FEE71B4B1C680725AC431C6017
:101DF0001C6814431C604368436043684360436845
:101E000043604368144C1C4044604368134C1C43BB
:101E100044600B0604681C43046003689B01FCD506
:101E200043680324A3434360436813434360426809
:101E30001207FCD5C806002130BC01F043BDC046E6
:101E4000001002400C00FF08FFFFC277FFFFF2FE08
:101E5000FF04000000200240FFFFC2F7000004085A
:101E600010B50A4C0121204601F060FF68B1012144
:101E7000204601F057FF0021204601F0B9FE04483A
:101E8000006810BC02BC8E46004710BD0020004018
:101E900014020020F8B51C4D01242846214601F00B
:101EA00045FF012803D10121284601F03BFF3649B7
:101EB00020310022154B164D032A10D09E5C5EB1D6
:101EC0000E460C3E37680868874201D2781C02E053
:101ED000AC54002098543060091D521CECE70D49A9
:101EE0000878294B58B19A68D868824202D2501CAF
:101EF000986004E0084804700020986008705968F1
:101F000009B1481E5860F8BD004001404102002060
:101F1000440200202F0200203002002010B5074CA0
:101F20000121204601F002FF012806D101212046AF
:101F300010BC04BC964601F0F5BE10BD0044014043
:101F4000B0B5104D01242846214601F0EFFE0128CE
:101F500003D10121284601F0E5FE0B480178022952
:101F600001D8491C02E009490C7000210170016987
:101F7000F02902D106490C7000214470491C01610E
:101F8000B0BDC04600480140F800002028020020F3
:101F900035020020B0B51D4C354D2046294601F0D4
:101FA0007BFF30B11A48006880472046294601F07F
:101FB0005FFF184D2046294601F03FFF012806D15A
:101FC0002046294601F031FF114800688047124D34
:101FD0002046294601F060FF30B110480068804774
:101FE0002046294601F044FF0D4D2046294601F0C8
:101FF00053FF48B109480068804720462946B0BCD5
:1020000004BC964601F034BFB0BDC0460038014064
:102010000C02002003070000070007071002002041
:1020200006000607B0B5114C114D2046294601F0B7
:1020300033FFD0B12046294601F01AFF0D48007841
:102040000D4D297881420BD2204601F0C5FE29783A
:102050000B4A50540B4801220270481C2870B0BD36
:1020600000202870054801210170B0BD00440040E7
:102070000500050728010020260100202501002079
:102080009801002024010020B0B5404800210171D2
:102090000424C4703C4D5A20A870EA206870A52022
:1020A00028702046FEF7BAFDE8702046B0BC02BC9E
:1020B0008E46FFF73BBEC046B0B5344800210171E3
:1020C0000424C470304DDC20A870EA206870A5207C
:1020D00028702046FEF7A2FDE8702046B0BC02BC86
:1020E0008E46FFF723BEC046400C0020B0B52748FF
:1020F000002101710424C470234DE520A870EA205A
:102100006870A52028702046FEF788FDE8702046FC
:10211000B0BC02BC8E46FFF709BEC04610B51A4AD5
:102120005070A5201070194C0220E070481C2071DE
:10213000FEF7F4FCE07810BC02BC8E46FFF7F6BD5B
:10214000BCB5114BA5241C70802404435C70009224
:10215000981C6A46521E0C4624B1155D0570401C41
:10216000641EF9E7094800220271C91CC170CCB293
:10217000E018451E2046FEF751FD28702046BCBCE5
:1021800002BC8E46FFF7D2BD400C00202401002087
:10219000B0B50020064CA047064D28600120A0479E
:1021A00068600220A047A8600320A047E860B0BD97
:1021B00031390008A801002010B5144608463F49EF
:1021C0000A220A700722214602F04AF8012804D1A7
:1021D000044802F0BFF8012801D0032010BD002000
:1021E00010BDC046204E0000F8B506460F4CA08832
:1021F000000A16D1A0880527032810D30D460092A7
:10220000A188264801F088FB48B924490878307035
:10221000481C2860A088801E009908800027384646
:10222000F8BD03A00C499C22FFF7C6FF1C0200204A
:102230007573526376427566666572506F73203CA3
:10224000204D425F5345525F5044555F53495A45B4
:102250005F4D415800000000814B0008B0B5174D9C
:102260006B780BB1052516E00124EC804B1EAB60AA
:102270001870E8888018E880E988184601F04CFB5F
:10228000E9884A1CEA80054A5054AC70002528466B
:10229000214601F047FE2846B0BDC0464A0C00204A
:1022A00010B501200024214601F03CFE0348447093
:1022B000204610BC02BC8E4601F0C0BF1C020020AC
:1022C00080B50020014601F02DFE80BC01BC864691
:1022D00001F05CBE10B5064C2078012805D10548F8
:1022E000806880470020207010BD062010BDC046C9
:1022F00014000020F4010020F8B50C4609880325DD
:1023000005292FD10279C17809028E18711E89B270
:10231000314B994226D8811C00918778417800255D
:1023200025800123037023885B1C23805307B2B2EE
:10233000D60803B1761C009B46702088401C208084
:102340000802C019401C81B218462B4600F0E8FA7A
:1023500020B1F8BC02BC8E4601F0BEBAF0B22188B2
:10236000081820802846F8BDF8B50C4609880325D2
:1023700005292ED10279C17809028E18711E89B201
:10238000154B994225D8811C00918778417800250A
:1023900025800223037023885B1C23805307B2B27D
:1023A000D60803B1761C009B46702088401C208014
:1023B0000802C019401C81B2184600F001FB20B190
:1023C000F8BC02BC8E4601F087BAF0B2218808182A
:1023D00020802846F8BDC046CE070000F8B50C4660
:1023E00009880325052923D10279511E7C291FD88C
:1023F000831C81784778002525800326067026886F
:10240000761C2680560046702088401C20803802AA
:102410004018401C81B218462B4600F0F7FA20B154
:10242000F8BC02BC8E4601F057BA20888019208083
:102430002846F8BDF8B50C4609880325052928D19A
:102440000179C278120251184A1E92B27B2A20D812
:10245000821C009287784378002525800422027030
:102460002288521C22808AB2560046702088401C66
:1024700020801802C019401C81B2009800F05CFB5B
:1024800020B1F8BC02BC8E4601F026BA2088801923
:1024900020802846F8BDF8B5054608880A2841D3AB
:1024A0000C462879E97809020F18781E80B20326B5
:1024B0007C2838D8287AE97909020818411E89B29F
:1024C000782930D8697A82B2500081422BD1A8791C
:1024D000697909020818411CA87800906E7828468E
:1024E0000A3089B2012300F091FAB0B9BAB23002D1
:1024F00000994018411CA81C0026268017232B7029
:1025000023885B1C238057006F7023885B1C23800B
:1025100089B2334600F07AFA38B1F8BC02BC8E4674
:1025200001F0DAB900263046F8BD2088C0192080B5
:10253000F9E70000B0B50C4605490D88401C891C20
:102540002A46FDF74DFE681C20800020B0BDC04625
:10255000C40100201CB50988032405291AD101797A
:10256000C1B982784378C178FF2900D091B91802A7
:102570008018421C01A800244470FF394B424B4193
:10258000037091B20122134600F0CAF910B101F0B4
:10259000A3F9044620461CBD80B50988052910D141
:1025A0008178427812025118491C89B2C01C01225C
:1025B000134600F02BFA30B180BC02BC8E4601F00D
:1025C0008BB9032080BD002080BD70B50C460A8801
:1025D0000321062A24D30679C27812029519AAB2D9
:1025E000D308760700D05B1C6D1EADB22D097A2D85
:1025F00016D84579DBB29D4212D1817843781B020F
:102600005918491C89B2801D012300F089F920B1B5
:1026100070BC02BC8E4601F05FB90520208000210D
:10262000084670BDB0B50C460A880321062A20D39F
:102630000279437955062D0EAB421AD1C3781B029D
:102640009A18531E9BB2772B13D8817843781B02BC
:102650005918491C89B2801D92B2012300F0D6F9A5
:1026600020B1B0BC02BC8E4601F036B905202080F6
:1026700000210846B0BD0000F8B50546022091B320
:10268000CC081E2C2FD8069C524E3170012D15D02F
:102690004DBB254D2548264FB760F0603561214878
:1026A00070611F48B0611D48F0611B4830620846E8
:1026B00011461A46234600F091F813E0134D1448D2
:1026C000144FB760F06035610F4870610D48B0611C
:1026D0000B48F06109483062084611461A46234605
:1026E000FFF76AFD00B1F8BD01F0A2FD20B1384846
:1026F000012101700020F8BD0320F8BDF940000859
:1027000031410008ED3F0008E92100085D22000882
:10271000C1220008A12200083D44000889440008A5
:10272000AD430008192800088D2800080D2900086D
:10273000F12800087CB52648007808B1062445E059
:1027400001A801F069FD002401283FD101A800780B
:10275000022812D0012839D11E4D6B69681C294608
:1027600024312A1D984788BB68782978884200D090
:1027700060BB022001F062FD28E0164D6A6A117804
:10278000A97000230120144C802B0AD0E65C46B1CE
:102790008E4201D00833F7E7E0184368291D104640
:1027A00098476978002489B158B10121A980A97896
:1027B00080220A43696A0A70A9884A1CAA806A6A48
:1027C0005054AA88696A28782B69984720467CBDAE
:1027D00014000020F40100201800002010B5144659
:1027E00008460822214601F03BFD01280ED144F69F
:1027F0000030844201D9232003E060000549B1FB89
:10280000F0F080B201F0A6FD012801D0032010BD38
:10281000002010BDA07F1700F8B506460F4C608859
:10282000000A16D160880527042810D30D460092AF
:1028300061882E4801F08EFA48B92C49087830702A
:10284000481C28606088C01E009908800027384610
:10285000F8BD03A00C499C22FFF7AEFCE801002064
:102860007573526376427566666572506F73203C6D
:10287000204D425F5345525F5044555F53495A457E
:102880005F4D415800000000234B0008B0B51E4DBD
:102890002B78012B26D10124AC804B1EAB60187025
:1028A000A8888018A880A988184601F053FAA9883A
:1028B0004A1CAA800D4A5054A9884B1CAB80000AC0
:1028C0005054A868007801F03BFDA888401EA880FD
:1028D000A868401CA8606C7000252846214601F0BD
:1028E00021FB00E005252846B0BDC0464A0C00206B
:1028F00080B5054800210170012001F013FB80BC68
:1029000001BC864601F05ABBE801002080B50020DA
:10291000014601F007FB80BC01BC864601F036BBD6
:10292000FEB514460246491E88B20019042824D870
:10293000601E0825019590FBF5F0451C0020F3B1C1
:10294000012B1BD100901D4B280435D06D1E029227
:1029500010782246019F541E12040BD03A0609D06B
:10296000012202408EB29A55491C7F1EC0B2400817
:102970002246F0E7029A521CE6E70120FEBD0090D5
:10298000082001900D4F280416D002926D1E0026DB
:1029900022460198541E12040AD0020608D08AB2B8
:1029A000BA5CB2401343761C491C401E2246F1E734
:1029B000029A1370521CE6E70098FEBD4A0D0020F3
:1029C000F0B5491E8BB2DC0801217D2C1BD39B186E
:1029D00040F2EC34A34216D8511E082391FBF3F1C8
:1029E0004C1C002125040ED0641E16461D46721E86
:1029F000360404D06F1E2D0616463D46F7D100253D
:102A00000570401CEEE70846F0BD0000FEB5054627
:102A1000481E87B2012002904148874217D91446C8
:102A2000BE18404A964212D841F27072BE1A3E4A0F
:102A30005660012B0DD033BB401C87424AD1022C7B
:102A400048D170003B490968384A115252E0029857
:102A5000FEBD019654700520C04340F2D07343433D
:102A60003248C0187B00C3182746164638040CD0DD
:102A70002878000218806A78801832461880AD1CC9
:102A80009B1C7F1EF2E70020FEBD41F2EB70081A8E
:102A900080B26B2802981CD801984000234909187D
:102AA0001078029047012248C519284608302206AE
:102AB000D20DFDF795FB01201D49C85101986860B2
:102AC0000298411CCAB200200F2A024600D80A46CA
:102AD0003270FEBD41F2EB70081A793080B2E32803
:102AE0000AD8700011490818B100124A5118620042
:102AF000FDF776FB002000E001200521CA4340F2EB
:102B0000D0715143094A5218790051182204E0D07B
:102B10004A782A700A786A70AD1C891C641EF5E731
:102B20006F170000581B0000B80100204E0D002058
:102B30003C0A00207C02002010B50346481E81B2EA
:102B40000120084CA1420BD38918074CA14207D899
:102B50000020110404D0587018709B1C521EF8E716
:102B600010BDC046B80B0000BC0B0000FCB50191C5
:102B7000016A0090446A00252E46202D0CD017468D
:102B8000F740FF0705D0019FAF400F23AB409943AB
:102B900039432D1D761CF0E708250026202E0CD089
:102BA0001346EB40DB0705D0019BB3400F27B7402E
:102BB000BC431C43361D6D1CF0E700980162446263
:102BC000FCBD8162704781617047C16270470069D6
:102BD0000840411E88417047FEB502930192026889
:102BE0000090C56800263746202E10D0029BFB407F
:102BF000DB0709D0019BB3400324B440A5431D4328
:102C00000B46B340A2431A43B61C7F1CECE7009866
:102C10000260C560FEBDF8B5012902D141681943C3
:102C200001E04168994341600090816800240320DD
:102C30002646202C0CD01F46F740FF0705D017462C
:102C4000A7400546A540A9433943A41C761CF0E7DC
:102C500000988160F8BD000000B59DB0EC4B0027E6
:102C60009F825F715F70EB480321189101700B2008
:102C7000C2431046093020B11918CF770F77401C96
:102C8000F9E71A921F72DF71FFF772F8FFF780FA07
:102C9000FEF752F9FEF7BAF9FEF730F9FEF700F940
:102CA000FEF74CF9FEF7C6FAFEF7D2F9FEF74EF83A
:102CB000FEF736FC42F28050FEF756FAFEF748F86F
:102CC0000920C006099001244020039080201C9018
:102CD0002546D0480078844226D8032C09D0022CFF
:102CE00011D0012C1ED1099E30460399FFF76BFFCE
:102CF0000EE0099E30460399FFF765FF30461C99A8
:102D0000FFF75FFF08E0099E30460399FFF759FF80
:102D100030461C99FFF757FFBF482946FFF753FF7E
:102D2000FEF7CAFA641CD4E7FEF774FD014600976B
:102D3000E120430238463A46FFF79EFCFFF7CAFA05
:102D400040F2F4213846B54F7A580399B04D6A5491
:102D5000B349E98140F60001C91C396040F2B41161
:102D60007958403501956970D1B20546FEF7C0FB30
:102D7000012109980591FFF724FF2524282C19D05B
:102D80000020A34908554819791940F2F8268A59B4
:102D90004423C25489198B6C46268355896F472377
:102DA000C154D1B220462438C0B2FEF7A1FB2D1D7C
:102DB000641CE3E740F21C3038582B21944E0891F4
:102DC000705407200C90C00340F2B41178500020DA
:102DD0000490F0728F4D1898287040F29430385853
:102DE00031462B31C87040F2643038588870308AD0
:102DF0007082059801040B9140040A90894940F2C1
:102E000006100818029040F2B8103818079040F2E7
:102E1000341008180690FDF777FE002800D00AE16C
:102E20000898325C1046059B18403073F17A88424E
:102E300003D10020B071317A24E0049C70B90123E1
:102E4000B3720021717252B2002A0BD53172F37144
:102E50002D22B25C40F2E8335A4310E0B472737230
:102E6000510604D433720022F271194607E034721D
:102E7000F3712D21725C40F2E8314A432146F07231
:102E80006948026039B300243472F471707A40B139
:102E900020216148FFF797FE74720898315C012089
:102EA0000AE0B07A60B120215B48FFF78AFEB47275
:102EB0000898315C1A980A30084340F21C31785067
:102EC000554C204644F20001FFF77DFE204644F2B7
:102ED0000001FFF776FE002716251C97192D00D15B
:102EE000A6E074193346F6194420315C01220846E5
:102EF0001B921040A074E27B824205D1585D00B362
:102F00000020434948551CE0002230B962721B9BE7
:102F1000237349B2002907D509E022731B9B637212
:102F2000490604D44149CA51E270A37108E0E37034
:102F3000A2714621715C40F2E83251433B4AD151C3
:102F4000E073A07900285BD0199744360027A77159
:102F5000E770607A58B17F201C990840022819D088
:102F6000012819D0E0B9099848F2000116E0207B49
:102F7000D0B327737F201C990840022817D001285E
:102F800017D0264C199FD0B9099848F20001FFF7D5
:102F900018FE14E0102100E008211F48FFF713FE7F
:102FA000677230781B9908431C4C199F0AE0102166
:102FB00000E008211848FFF704FE184C199F3078EC
:102FC0001B99884329461639E219C0B240F2F8230A
:102FD000D050CAB2189BB2FBF3F25A43891A363961
:102FE000CF220A40910060500B4C204644F2000171
:102FF000FFF7E9FD204644F20001FFF7E2FD199FCB
:103000006D1C3F1D1C98401C1C90014E66E7C0467D
:103010002802002000000020000400487C0200205C
:10302000030800001C0700200401002018010020F4
:1030300000207080EC4FFFF77DFBFDF7D1FD18B14C
:10304000FEF74EFAFDF776FD707BF8B10020707345
:103050001A98A0B1E54909183A18526B40F2431387
:10306000CA54130A40F242140B55130C40F2411497
:103070000B55120E40F24013CA54001DE9E740F20E
:1030800005102F300C220699FDF7AAFC3078002895
:1030900000D11CE200243470032C04D0E0B200F014
:1030A000FBFC641CF8E7D24C206A1990606A15900A
:1030B000A06A1490236C656CA06C13902246603259
:1030C00007CA1292199A7A601793BB601690F8603B
:1030D0001598386111957D61C64D1091B9611498AC
:1030E000F861139838623246343207CAA36B1B1852
:1030F000A06D4118A06F8018129A7A620F93BB627C
:103100000E91F9620D90386340F2B413FC180D264D
:10311000112E00D1CBE11C9430460D38AC191A9910
:10312000615CC0001B90F1B10D2E23D140F2B415AB
:1031300040F2E810385801230027199981421946B6
:1031400000D83946A84A5559189A95436918179ACC
:10315000824200D83B465B00C918169A82421FD9AA
:10316000042001431EE00D2E14D1F8580C99884319
:10317000F85028E01B980D3080B2800039581C9A16
:10318000906C814214D910680121014302208143CF
:10319000116018E01C9A106801218843106012E049
:1031A00004208143904F40F2B413F950914D0AE04E
:1031B0001068189B9843936F994201D802210843E5
:1031C000106040F2B4131A980419E07890B10D2EF3
:1031D00025D1384640F2EC117F58C158864830302E
:1031E0000840199BBB4246D840F2E8318B423FD998
:1031F00008213FE00D2E1FD1FF587F48074040F2C5
:10320000E8301999814202D848F20000074340F2A1
:10321000E830179981421BD80B9807431AE01B9896
:103220000D3080B2800039581C9A1068936C994216
:1032300008D90221884307E01C9A106802218843BC
:1032400010603DE002210843106040F2B41337E003
:103250006A48074040F2E8301699814202D968482E
:10326000074001E00A9807435F48C750074627E038
:1032700048F200010843614B283303401798B842D5
:1032800008D8014640F2E830814201D9102000E020
:103290000B9803435A4818301840169BBB4203D979
:1032A000514F40F2B4130AE040F2E8318B424E4FE6
:1032B00040F2B41301D9202100E00A990843F850E4
:1032C000A07900B30D2E26D13946FF58C020874380
:1032D00040F2F010085801210025159B83420B464F
:1032E00000D82B469B01FF18119B834200D829462A
:1032F000C9017918109B834240F2B4131FD940F2E0
:10330000001001431EE00D2E13D1F8583D4926311F
:103310000140F9501FE0A8201C9A11581B980E304C
:1033200080B280003B5810688B420FD904210843BB
:103330000EE01C9A10680421884310600BE03148AD
:10334000E6300140284FF9502A4D04E0042188431B
:10335000106040F2B413607A80B10D2E17D140F2A4
:10336000B4103B5840F20060834340F2F4103858E8
:103370000024149981421DD821461CE00D2E1C9C6E
:1033800013D1F85840F600618843F85043E0D82044
:103390001C9C21581B980F3080B280003B5820683D
:1033A0008B421BD9082108431AE020680821884372
:1033B000206030E0012149025B181399814202D953
:1033C00040F2E8341834234340F2B4117B50129C8D
:1033D000844219D940F60000034318E008218843CD
:1033E000206040F2B41316E07C0200201C0700208D
:1033F0007C06002000000020C77FFFFFC7FFFEFF04
:10340000C7FFFDFF19FEFFFF40F6000083437B501E
:1034100040F2B4131C9CA85D10B30D2E28D1F958AE
:1034200043F20000814340F2F41038580123002495
:103430000F9D85421D4600D825462D0349190E9D36
:10344000854200D823465B03C91840F2B413F950F3
:103450000D9C8442FA4D44F200001CD901431BE04C
:103460000D2E13D1F85847F200018843F8501BE0A5
:1034700040F2081021581B98103080B280003B5851
:1034800020688B420BD9102108430AE020681021E4
:103490008843206008E08143F9501C9C04E010211F
:1034A0008843206040F2B413241D761C30E6E34EBE
:1034B000308A0021079A032908D001238B4010CAC3
:1034C0000CB1184300E09843491CF4E7308270794E
:1034D0004101DF4B5A58002A00D182E05818446855
:1034E0007A2C78D321467A3904291CD88A0001A382
:1034F0009A18974600F008B800F02BB800F038B8DA
:1035000000F046B800F054B8806840F2E8117850F6
:10351000CE4A1071010AD170010C9170000E5070EA
:10352000511C012053E08A2C03D9962C01D9A22CDE
:103530005FD88068A1007850C34A8A18010EC34B37
:1035400099549918C870030C4B70000A887090B297
:103550003DE0806840F2EC117850BC4A1072010ADC
:10356000D171010C9171000E5071511D05202EE09A
:10357000806840F2F0117850B44A1073010AD17299
:10358000010C9172000E50721146093109201EE0A3
:10359000806840F2F4117850AC4A1074010AD1737B
:1035A000010C9173000E507311460D310D200EE089
:1035B000806840F2F8117850A44A1075010AD1745D
:1035C000010C9174000E5074114611311120042227
:1035D000FDF706FA9E4B7079410100225A500121F5
:1035E0003171401CC1B20F2900D900207071FFF762
:1035F00012FCAE2C11D8A100934A5218934D5319C6
:1036000080683324185578503032010EA954010CCB
:1036100031241955000A322112E0BA2C13D8A10026
:10362000894A5218894D5319806863241855785077
:103630006032010EA954010C61241955000A62215F
:103640005854A91883E7BD2C14D0BC2C26D0BB2C11
:1036500048D10125B5707D4840F20611401844213B
:10366000502949D002784123134373540370091D34
:10367000801CF5E78068039C305540F20511734AC1
:10368000505440F2F4217850C1B240F20510FDF7D9
:10369000B7F9315D0020FDF72BFF9BE70120F070AB
:1036A0004420029950280AD00A787E2313407F22B2
:1036B000D2439A1832540A70001D891CF2E7634CF9
:1036C00040F20610211840F20510401C0622FDF7BA
:1036D00087F940F21812A05C7E2101407F20C04390
:1036E000081817E0C92C1ED8017A2546BE3D092DC1
:1036F0005ED10898315468E0544C40F2061021180D
:1037000040F20510401C0622FDF76AF940F218123B
:10371000A05C284308997054A054A11840F20510E9
:103720001330022254E7CF2C59D88168CA3C18982C
:103730006043421C9300019DE954871CBE00A955BB
:10374000C01C1C9080001B9029543C480019012388
:103750008375D0B2C9B23F4A9047A95DF8B2394FDC
:103760003C4EB04732461B98295C344E1C98C0B280
:1037700090470620604340F200110C18A01D71799B
:103780004901334A5118097A304A115425460835FF
:1037900051550A34115580B22F4A90472B48415D4C
:1037A000A8B22D4DA8472948015DA0B2A84711E74E
:1037B000BD3CA0003018039A8154E0B21C46FDF7CE
:1037C00097FE7079400120188168680040F200126D
:1037D0001018801D1D4A115480B2C9B22BE0DB2C99
:1037E0000ED8826820464E3018490A54D1B2A30040
:1037F000F950D92C16D09B1940F2FA241B1B13E068
:10380000E52C00D9E7E6806822464E320F498854FD
:10381000C1B2A300F950E52C09D09B1940F229341C
:103820001B1B06E033462D331A7080B203E033468B
:103830002E33187090B2FDF7E3F8CBE62802002093
:10384000000000207C02002019FEFFFF1C07002062
:103850003C0A0020F1140008010A000870B540B2CB
:10386000002817D4032302469A43144BD4588507E3
:10387000ED0EFF26AE40B4438901C9B2A9402143F1
:10388000D1501F21014001228A40400980000C498B
:10389000425070BD8207D20EFF2494400F23034094
:1038A000083B0320834304481D58A5438901C9B23E
:1038B00091402943195070BD1CED00E000E400E088
:1038C00000E100E0024A0A400243024802607047F9
:1038D00080FFFF1F08ED00E040B1072803D001285A
:1038E00003D1022070470620704704207047000073
:1038F0000A2801D2302102E0102803D2372108180B
:10390000C0B2704702A0034940F2D012FEF754FC47
:1039100030000000814B000800220B0405D0037822
:10392000D218D2B2401C491EF7E75042C0B27047CD
:10393000F8B501463E4B18680C2202403D48082A63
:10394000044618D11A689202120F0F2A01D0941C53
:1039500000E010241D682D0101D5113214461A68AB
:10396000D20301D4344A05E09A6A0F2515406A1C37
:10397000B0FBF2F254431D6818681A6805291FD875
:1039800000902D062D0F2DA77F5D2546FD4092044A
:10399000520F2E4FBE5C2A46F2408E0001A08019C5
:1039A0008746C04600F00AB800F011B800F00AB827
:1039B00000F00EB800F00EB800F014B8224607E090
:1039C000002205E000984005400F385CC5402A46BB
:1039D0001046F8BDD86AC0051AD4D86AC00320D5ED
:1039E0001C48F8BDD86A8007F2D0D86A0321084085
:1039F00001282246ECD0D86A084048F2000202288A
:103A0000E6D0D86A084003280A4800D00020F8BD54
:103A100018680004800FD96A002904D4B2FBF0F2C0
:103A2000D6E70B48F8BD401CB5FBF0F2D0E7C04626
:103A30000410024000127A0000093D00000000005E
:103A4000000000000102030406070809B84A000844
:103A5000809FD500003FAB011F21014001228A4019
:103A600080090C4943581343435070471F210140BC
:103A700001228A40800907494358934343507047C5
:103A80001F21014001228A40800902494358134303
:103A90004350704700100240FEB50446401C4F4F93
:103AA000B871022C0CD0012C16D0002C00D094E060
:103AB00002900920C50640212846FFF784F812E04D
:103AC00002900920C50640212846FFF77CF8802196
:103AD0002846FFF776F80AE002900920C506402143
:103AE0002846FFF76EF880212846FFF76CF83C481F
:103AF0000121FFF768F8FCF7A3FFB86C394D2946A0
:103B000000F0FAFDFCF7ECFD1F2800D20020B97987
:103B10004901354A50505618386C294600F0ECFDE2
:103B2000FCF7DEFD70601E2804D8301D00250560FE
:103B300028460CE0386D2B4900F0DEFDFCF7D0FD87
:103B40000546786D274900F0D7FDFCF7C9FDE10077
:103B500001913061B5606DB1386DFC6E2146FCF7A6
:103B60000FFD796D00F020FE1E4900F0C5FDFCF749
:103B7000B7FD01E0FC6E0020F060B86E194D2946DB
:103B800000F0BAFDFCF7ACFD7061386E294600F01C
:103B9000B3FDFCF7A5FDB0612046294600F0ACFD61
:103BA000FCF79EFDF061029840010F490A5802920D
:103BB000019AD2B292000D4BD2180818071DF8CF07
:103BC0008169C0690190029850639363D46315645E
:103BD00056649764D16401981065FEBD24010020ED
:103BE0000004004800007A447C0600207C0200208B
:103BF0004162704710B5154C4449884213D01449AE
:103C0000884212D0EC49884211D03D49884213D0F5
:103C10003D4988420DD03E4988420CD039498842FE
:103C200013D1F63408E0E41D06E0F93404E0FD3475
:103C300002E0641D00E0A41D2046FFF721FF20469E
:103C400010BC02BC8E46FFF711BF10BD0B03000075
:103C50000010004001680122914301607047016833
:103C600001220A430260704710B50A888262244A22
:103C7000904202D0234B98420BD103687024A34397
:103C800003604B8804681C4304608B8804681C43F1
:103C900004608B68C36290420FD1136840F2003415
:103CA000A3431360CB8814681C431460097B016331
:103CB000416901220A43426110BD124A90420BD071
:103CC000C94A904208D0104A904205D00F4A90420B
:103CD00002D00F4A9042EBD1026840F200339A437F
:103CE0000260CA88036813430360074A9042DDD02C
:103CF000074A9042DAD0054A9042D7D0D8E7C0466A
:103D0000002C0140000400400040014000480140F8
:103D100000440140C2688A43C2607047C2680A43D7
:103D2000C260704702698A4302617047C2680A40F4
:103D3000531E9A4100690840411E88411040704757
:103D40000349002202730260426081607047C046EE
:103D5000FFFF0000F0B5FF24094A0A4B25460E0478
:103D600009D006787540565D5F5D25467D40401C54
:103D7000491E3446F3E72002284380B2F0BDC04616
:103D8000B8490008B8480008B0B50D4604467E485A
:103D9000844204D02048844205D1022000E005205E
:103DA000FFF7C6FD00E000202168090405D469087A
:103DB0004018B0FBF5F080B209E0690840004018F7
:103DC000B0FBF5F0034901400007400F4018E060E8
:103DD000B0BDC046F0FF0000416A0348084070478C
:103DE000014A0A4082627047FF01000010B566492F
:103DF000884204D0084988420BD1084C00E0054CA9
:103E00002046FFF73DFE204610BC02BC8E46FFF761
:103E10002DBE10BD0E030000004400401104000040
:103E2000016801220A43026070471F220A400121F3
:103E30009140026A0A43026270471F220A408909C0
:103E40000958D1400120084070471F220A40012331
:103E5000934089090A589A430A5070471F220A4022
:103E60000123934089090A581A430A5070470000F9
:103E7000084A914206D1D021425848F200039A43A1
:103E800042507047C902C90E01228A40016A11439B
:103E90000162704709340F341F220A400B049B0D46
:103EA0001B58D3408A0D1258C802C00EC2401A4097
:103EB000012010407047026801239A4302600268A3
:103EC00040F200639A43026002680A43026070474E
:103ED000026804239A43026002680A430260704742
:103EE000026801239A430260426843F200039A4346
:103EF000426042680A4342607047026808239A435E
:103F0000026002680A4302607047026801239A4314
:103F10000260026841F200039A43026002680A43A9
:103F20000260704770B50E460921CC06CB4D0521C5
:103F3000012808D12846FFF791FF204640F60001EE
:103F4000FEF73FFE07E02846FFF77FFF204640F6DA
:103F50000001FEF738FE06212846012E09D1FFF7A1
:103F60007DFF204640F6000170BC04BC9646FEF77B
:103F70002ABEFFF76AFF204640F6000170BC04BC71
:103F80009646FEF71EBEC04600380140B0B5164C3E
:103F900000212046FFF72CFE012520462946FFF789
:103FA000C1FE20462946FFF7B5FE2046B0BC02BC44
:103FB0008E46FFF74FBEC04600200040B0B50A4C09
:103FC00000212046FFF714FE012520462946FFF771
:103FD000A9FE20462946FFF7A1FE2046B0BC02BC40
:103FE0008E46FFF73CBEC04600200040BCB53A4DAF
:103FF000A87800286AD101A800F028F96878002480
:1040000078B1022818D001285ED1FFF7D7FF01A8A8
:1040100000780D2828D000243A2828D1EC70AC80F4
:1040200052E001A800783A284ED1FFF7C7FF0024DC
:10403000AC80EC70012018E001A800782978884253
:1040400008D1FFF7A3FF00206870012000F0F6F808
:10405000044639E000243A2810D1EC70AC800120ED
:104060006870FFF7ABFF2FE0022068702CE001467C
:104070004139C9B2062903D3E14303E06C7023E060
:10408000014637393038C2B20A2A00D30846E978E7
:1040900001290AD0C1B9A988FF2911D8A98800012E
:1040A000E54A50540120E8700EE0A988E24A535CCA
:1040B00003435354A888401CA8800024EC7003E0FC
:1040C00000246C70FFF762FF2046BCBD03A051497D
:1040D000E322FEF771F8C0461C02002065536E64AF
:1040E0005374617465203D3D2053544154455F54E1
:1040F000585F49444C45000080B53E484178491E10
:10410000012902D80021417005E04178012902D03F
:104110004078022803D1FFF739FF002080BD034813
:104120003C4940F2A712FEF747F8C0463D4B000855
:1041300070B5304E7078002856D1B078042840D839
:10414000810001A251188F4600F008B800F027B88E
:1041500000F009B800F02BB800F014B801200021DD
:10416000FFF7E0FE2DE0F08830B3F07801282AD088
:1041700038BBB06800780009FFF7BAFB00F0E0F840
:10418000012012E00024B470032000F057F8054627
:1041900001202146FFF7C6FEB470284670BD3A20C4
:1041A00000F0CEF80220B0700020F07009E0307806
:1041B00000F0C6F8042003E00D2000F0C1F8032051
:1041C000B070002070BDB06801780F200840FFF784
:1041D0008FFB00F0B5F80020F070B068401CB060B4
:1041E000F088401EF080ECE703A00A4940F24F122D
:1041F000FDF7E2FF1C020020655263765374617480
:1042000065203D3D2053544154455F52585F494419
:104210004C450000814B00080B490A78012A05D162
:104220004A78027000200870012070470020704713
:1042300005480021017001207047C04602494870BE
:10424000012008707047C046C001002010B5044628
:104250003F48FFF7C1FD2070012010BD003801402C
:10426000FEB502911B2000252946FFF7F7FA3148D9
:10427000FFF7F2FB0920C60601243046214640F232
:104280000022FEF773FC022101913046224640F2E3
:104290000023294FB847294F30462946224640F28D
:1042A0000023B8473046214640F20042FEF75EFC4C
:1042B00030460199224640F200431F4FB84730462E
:1042C0002946224640F200431C4FB847304621465B
:1042D0002A4640F60003184FB847032230462946C5
:1042E00040F60003154EB0471248FD30FFF7B4FB0F
:1042F000174E3046FFF77AFD30460299FFF744FD2E
:1043000030462946FFF7ECFD30462946FFF7FDFD14
:1043100030462946FFF7CFFD04213046FFF7D8FD90
:1043200008213046FFF7E9FD3046FFF779FD2046CA
:10433000FEBDC04611050000D92B0008172C00084F
:1043400080B501460248FFF74BFD012080BDC04605
:10435000003801407FB5054640F20870FFF77CFB4E
:10436000104C2046FFF746FC6E463046FFF7E8FC4F
:104370000D483080681E0290002001902046314692
:10438000FFF772FC012520462946FFF7C7FC1320E2
:104390002946FFF763FA2046FFF761FC284604B080
:1043A00070BDC046002000400F0E00001CB51A4C26
:1043B000607858BB01A8FFF749FF2078032823D86D
:1043C000810001A251188F4600F01CB800F004B81B
:1043D00000F00CB800F016B8002060806088411C26
:1043E00061801549019A0A5402200AE06088FF287A
:1043F00006D86088411C61800F49019A0A5401E087
:1044000003202070FFF7DAFD00201CBD03A03D490A
:10441000F022FDF7D1FEC046E801002065536E642E
:104420005374617465203D3D2053544154455F549D
:10443000585F49444C4500004A0C0020B0B5294D56
:1044400028780024032808D0022802D058B9002078
:1044500000E00120FFF7F2FE0446FFF797FD012080
:1044600028702046B0BD28780028F6D02878022889
:10447000F3D028780328F0D00248224940F2651290
:10448000FDF79AFEC04A000870B5164E3078012834
:1044900022D17078012805D080B901200021FFF7D2
:1044A00041FD0BE0B08858B1B0680078FFF748FFD5
:1044B000B068401CB060B088401EB080002070BD65
:1044C0000320FFF7BBFE0446012000252946FFF725
:1044D00029FD7570204670BD03A00A4940F22B12D9
:1044E000FDF76AFEE801002065526376537461743B
:1044F00065203D3D2053544154455F52585F494427
:104500004C450000234B000810B500F029F8EFF3EC
:104510000080800001D4012010BD002010BD10B526
:1045200000F096F8EFF30080800001D5012010BD67
:10453000002010BD10B500F08BF8EFF300804000B4
:10454000800F012800D0002010BD10B500F0AAF89F
:10455000EFF30080800001D4012010BD002010BDC9
:1045600070B501252D050C001C4310D4EC4206D477
:10457000AC420AD4994200D070BD904270BDE9426D
:1045800017D4EB4215D4994270BD894270BDEC42FC
:1045900006D5AC42F9D58B4200D070BD824270BDC9
:1045A0006D004C00EC4204D25C00EC4201D28B4224
:1045B00070BD034C30B4FCF7DBF830BC70BD00BFFD
:1045C0001900160470B50125ED0704004C4020D4F5
:1045D000441A01D2001B0919C60D4B00F2B2FF2A82
:1045E00029D01B0E2CD000020C0228432C43D31AD6
:1045F000DC40051910D2280A02D3401C6D0611D0E8
:10460000761EF6058019FF2A00DA70BDC00DC005C0
:1046100070BD694000F0CEF801200543C541521C31
:10462000761CE8E764089C40C90161408900E7D135
:104630000124A043E4E71B0E440200D0034870BDF0
:10464000002AFCD1C00FC00770BD00BF0000C07FB2
:104650000123DB0502000A430DD4DA4203D49A4257
:1046600007D488427047D84214D4D94212D4884221
:10467000704780427047DA4203D59A42F9D58142A9
:1046800070475B004200DA4204D24A00DA4201D2AB
:104690008142704710B5024AFCF7BAF810BD00BF5E
:1046A000090013040123DB0502000A430DD4DA429A
:1046B00003D49A4207D488427047D84214D4D942CE
:1046C00012D48842704780427047DA4203D59A423A
:1046D000F9D5814270475B004200DA4204D24A00B9
:1046E000DA4201D28142704710B5024AFCF790F8D5
:1046F00010BD00BF0900160470B5420064414B00B4
:104700005C41120E39D01B0E38D0FF2A3CD0FF2B53
:104710003AD0D2187F3A40024902400A490A451865
:10472000ED0106004E43000A090A48430104731ACA
:104730004019190C4318990F04D05B08012149074F
:104740005B1A521CD80904D3401CF50301D19D0605
:1047500007D0FF2A08D2D50506D0E4072043401928
:1047600070BD0125A843F4E7002A01DCE00770BD15
:104770002402FF202043C00570BD1B0EFF2A03D07A
:10478000FF2B01D0E00770BDFF2636064500B5427D
:1047900006D84D00B54203D8D218FF2A00D0E7E76B
:1047A000004870BD0000C07F70B50125ED07040012
:1047B0004C4022D4441A02D26C40001B0919C60D89
:1047C0004B00F2B2FF2A4BD01B0E50D000020C025D
:1047D000A8432C43D31ADC40051B05D5AD0019D3E3
:1047E0006D08761E521E37D0F605280A01D28019B0
:1047F00070BD70416D0603D070BD6940FFF7E8FEE3
:104800009C4009026140490001D0401E70BD012456
:10481000A04370BD6D081DD001202B0C01D12D04CB
:1048200010302B0E01D12D0208302B0F01D12D019C
:10483000001DAB0F01D1AD00801CEB0F01D16D004D
:10484000401C361A121A6D00680AF5054019012A33
:1048500002DB70BD002070BDC036300AC00770BDDD
:104860001B0E440201D1FF2B00D1024870BD002A6B
:10487000F0D070BD0000C07F8182838485868788E8
:10488000898B8C8D8E8F919293959697999A9C9DFA
:104890009FA0A2A3A5A7A8AAACAEB0B2B3B5B7B962
:1048A000BCBEC0C2C5C7C9CCCED1D4D7D9DCDFE22B
:1048B000E6E9ECF0F3F7FAFE00C1814001C0804167
:1048C00001C0804100C1814001C0804100C18140E0
:1048D00000C1814001C0804101C0804100C18140D0
:1048E00000C1814001C0804100C1814001C08041C0
:1048F00001C0804100C1814001C0804100C18140B0
:1049000000C1814001C0804100C1814001C080419F
:1049100001C0804100C1814000C1814001C080418F
:1049200001C0804100C1814001C0804100C181407F
:1049300000C1814001C0804101C0804100C181406F
:1049400000C1814001C0804100C1814001C080415F
:1049500001C0804100C1814000C1814001C080414F
:1049600001C0804100C1814001C0804100C181403F
:1049700000C1814001C0804100C1814001C080412F
:1049800001C0804100C1814001C0804100C181401F
:1049900000C1814001C0804101C0804100C181400F
:1049A00000C1814001C0804100C1814001C08041FF
:1049B00001C0804100C1814000C0C101C30302C2E7
:1049C000C60607C705C5C404CC0C0DCD0FCFCE0E4F
:1049D0000ACACB0BC90908C8D81819D91BDBDA1ABF
:1049E0001EDEDF1FDD1D1CDC14D4D515D71716D62F
:1049F000D21213D311D1D010F03031F133F3F2329F
:104A000036F6F737F53534F43CFCFD3DFF3F3EFE0E
:104A1000FA3A3BFB39F9F83828E8E929EB2B2AEA7E
:104A2000EE2E2FEF2DEDEC2CE42425E527E7E626EE
:104A300022E2E323E12120E0A06061A163A3A2625E
:104A400066A6A767A56564A46CACAD6DAF6F6EAECE
:104A5000AA6A6BAB69A9A86878B8B979BB7B7ABA3E
:104A6000BE7E7FBF7DBDBC7CB47475B577B7B676AE
:104A700072B2B373B17170B050909151935352921E
:104A800096565797559594549C5C5D9D5F9F9E5E8E
:104A90005A9A9B5B99595898884849894B8B8A4AFE
:104AA0004E8E8F4F8D4D4C8C44848545874746866E
:104AB00082424383418180400000000001020304E0
:104AC0002820655263765374617465203D3D205300
:104AD000544154455F52585F494E49542029207C27
:104AE0007C202820655263765374617465203D3DB7
:104AF0002053544154455F52585F52435620292059
:104B00007C7C202820655263765374617465203D57
:104B10003D2053544154455F52585F4552524F52C5
:104B20002029002E2E2F4170702F4D6F64627573F7
:104B30002F7274752F6D627274752E630028206554
:104B40005263765374617465203D3D205354415443
:104B5000455F52585F5243562029207C7C202820F4
:104B6000655263765374617465203D3D2053544112
:104B700054455F52585F574149545F454F4620297D
:104B8000002E2E2F4170702F4D6F646275732F6150
:104B9000736369692F6D6261736369692E630000D5
:104BA000C04B000800000020980000001001000821
:104BB000584C000898000020881C00002C010008B8
:104BC00003010000010000010000010000010000DD
:104BD00000A24A0402000000110000003525000870
:104BE000040000003524000803000000DD23000855
:104BF0001000000025260008060000009925000886
:104C0000170000009724000801000000F9220008A6
:104C100005000000552500080F000000CB25000806
:104C200002000000692300080000000000000000EE
:104C30000000000000000000000000000000000074
:104C40000000000000000000000000000000000064
:084C500000000000000000005C
:04000005080001A945
:00000001FF
